 retransform004

 Timestamp is 12c99756 (reproducible build file hash)

 Preferred load address is 0000000180000000

 Start         Length     Name                   Class
 0001:00000000 00002e40H .text$mn                CODE
 0001:00002e40 00000036H .text$mn$00             CODE
 0001:00002e76 00000092H .text$x                 CODE
 0002:00000000 00000190H .idata$5                DATA
 0002:00000190 00000038H .00cfg                  DATA
 0002:000001c8 00000008H .CRT$XCA                DATA
 0002:000001d0 00000008H .CRT$XCZ                DATA
 0002:000001d8 00000008H .CRT$XIA                DATA
 0002:000001e0 00000008H .CRT$XIC                DATA
 0002:000001e8 00000008H .CRT$XIZ                DATA
 0002:000001f0 00000008H .CRT$XLA                DATA
 0002:000001f8 00000008H .CRT$XLZ                DATA
 0002:00000200 00000008H .CRT$XPA                DATA
 0002:00000208 00000008H .CRT$XPZ                DATA
 0002:00000210 00000008H .CRT$XTA                DATA
 0002:00000218 00000008H .CRT$XTZ                DATA
 0002:00000220 00000000H .gehcont$y              DATA
 0002:00000220 00000000H .gfids$y                DATA
 0002:00000220 00001be0H .rdata                  DATA
 0002:00001e00 00000000H .rdata$CastGuardVftablesA DATA
 0002:00001e00 00000000H .rdata$CastGuardVftablesC DATA
 0002:00001e00 00000028H .rdata$T                DATA
 0002:00001e28 000000a8H .rdata$voltmd           DATA
 0002:00001ed0 00000320H .rdata$zzzdbg           DATA
 0002:000021f0 00000008H .rtc$IAA                DATA
 0002:000021f8 00000008H .rtc$IZZ                DATA
 0002:00002200 00000008H .rtc$TAA                DATA
 0002:00002208 00000008H .rtc$TZZ                DATA
 0002:00002210 00000004H .tls                    DATA
 0002:00002214 00000004H .tls$                   DATA
 0002:00002218 00000008H .tls$ZZZ                DATA
 0002:00002220 00000330H .xdata                  DATA
 0002:00002550 000003c4H .edata                  DATA
 0002:00002914 00000064H .idata$2                DATA
 0002:00002978 00000018H .idata$3                DATA
 0002:00002990 00000190H .idata$4                DATA
 0002:00002b20 00000414H .idata$6                DATA
 0003:00000000 00000080H .data                   DATA
 0003:00000080 0001b238H .bss                    DATA
 0004:00000000 00000390H .pdata                  DATA

  Address         Publics by Value              Rva+Base               Lib:Object

 0000:00000000       __AbsoluteZero             0000000000000000     <absolute>
 0000:00000000       ___safe_se_handler_count   0000000000000000     <absolute>
 0000:00000000       ___safe_se_handler_table   0000000000000000     <absolute>
 0000:00000000       __arm64x_extra_rfe_table   0000000000000000     <absolute>
 0000:00000000       __arm64x_extra_rfe_table_size 0000000000000000     <absolute>
 0000:00000000       __arm64x_native_entrypoint 0000000000000000     <absolute>
 0000:00000000       __arm64x_redirection_metadata 0000000000000000     <absolute>
 0000:00000000       __arm64x_redirection_metadata_count 0000000000000000     <absolute>
 0000:00000000       __dynamic_value_reloc_table 0000000000000000     <absolute>
 0000:00000000       __enclave_config           0000000000000000     <absolute>
 0000:00000000       __guard_check_icall_a64n_fptr 0000000000000000     <absolute>
 0000:00000000       __guard_eh_cont_count      0000000000000000     <absolute>
 0000:00000000       __guard_eh_cont_table      0000000000000000     <absolute>
 0000:00000000       __guard_fids_count         0000000000000000     <absolute>
 0000:00000000       __guard_fids_table         0000000000000000     <absolute>
 0000:00000000       __guard_iat_count          0000000000000000     <absolute>
 0000:00000000       __guard_iat_table          0000000000000000     <absolute>
 0000:00000000       __guard_longjmp_count      0000000000000000     <absolute>
 0000:00000000       __guard_longjmp_table      0000000000000000     <absolute>
 0000:00000000       __hybrid_auxiliary_iat     0000000000000000     <absolute>
 0000:00000000       __hybrid_auxiliary_iat_copy 0000000000000000     <absolute>
 0000:00000000       __hybrid_code_map          0000000000000000     <absolute>
 0000:00000000       __hybrid_code_map_count    0000000000000000     <absolute>
 0000:00000000       __x64_code_ranges_to_entry_points 0000000000000000     <absolute>
 0000:00000000       __x64_code_ranges_to_entry_points_count 0000000000000000     <absolute>
 0000:00000100       __guard_flags              0000000000000100     <absolute>
 0000:00000000       __ImageBase                0000000180000000     <linker-defined>
 0001:00000000       ?NewObject@JNIEnv_@@QEAAPEAV_jobject@@PEAV_jclass@@PEAU_jmethodID@@ZZ 0000000180001000 f i libretransform004.obj
 0001:00000028       ?SetEventNotificationMode@_jvmtiEnv@@QEAA?AW4jvmtiError@@W4jvmtiEventMode@@W4jvmtiEvent@@PEAV_jobject@@ZZ 0000000180001028 f i libretransform004.obj
 0001:00000034       ?TranslateError@@YAPEBDW4jvmtiError@@@Z 0000000180001034 f   libretransform004.obj
 0001:000002ec       ?nsk_jni_check_exception@@YAHPEAUJNIEnv_@@QEBDH@Z 00000001800012ec f   libretransform004.obj
 0001:00000430       ?nsk_jni_lverify@@YAHHPEAUJNIEnv_@@HQEBDH1ZZ 0000000180001430 f   libretransform004.obj
 0001:000004d0       Agent_Initialize           00000001800014d0 f   libretransform004.obj
 0001:00000740       Agent_OnAttach             0000000180001740 f   libretransform004.obj
 0001:00000740       Agent_OnLoad               0000000180001740 f   libretransform004.obj
 0001:00000818       Java_nsk_jvmti_RetransformClasses_retransform004_forceLoadedClassesRetransformation 0000000180001818 f   libretransform004.obj
 0001:000008a8       Java_nsk_jvmti_unit_FollowReferences_FollowRefObjects_addRefToVerify 00000001800018a8 f   libretransform004.obj
 0001:00000a80       Java_nsk_jvmti_unit_FollowReferences_FollowRefObjects_getTag 0000000180001a80 f   libretransform004.obj
 0001:00000b40       Java_nsk_jvmti_unit_FollowReferences_FollowRefObjects_resetRefsToVerify 0000000180001b40 f   libretransform004.obj
 0001:00000b48       Java_nsk_jvmti_unit_FollowReferences_FollowRefObjects_resetTags 0000000180001b48 f   libretransform004.obj
 0001:00000b8c       Java_nsk_jvmti_unit_FollowReferences_FollowRefObjects_setTag 0000000180001b8c f   libretransform004.obj
 0001:00000de4       Java_nsk_share_jvmti_ArgumentHandler_getAgentOptionsString 0000000180001de4 f   libretransform004.obj
 0001:00000e94       Java_nsk_share_jvmti_DebugeeClass_checkStatus 0000000180001e94 f   libretransform004.obj
 0001:00000f1c       Java_nsk_share_jvmti_DebugeeClass_resetAgentData 0000000180001f1c f   libretransform004.obj
 0001:00000f7c       Java_nsk_share_jvmti_RedefineAgent_agentStatus 0000000180001f7c f   libretransform004.obj
 0001:00000f88       Java_nsk_share_jvmti_RedefineAgent_isRedefined 0000000180001f88 f   libretransform004.obj
 0001:00000f94       Java_nsk_share_jvmti_RedefineAgent_redefineAttempted 0000000180001f94 f   libretransform004.obj
 0001:00000fa0       MA_checkStatus             0000000180001fa0 f   libretransform004.obj
 0001:00001044       __local_stdio_printf_options 0000000180002044 f i libretransform004.obj
 0001:00001224       exitOnError                0000000180002224 f   libretransform004.obj
 0001:000012d8       fprintf                    00000001800022d8 f i libretransform004.obj
 0001:0000131c       nsk_jvmti_createJVMTIEnv   000000018000231c f   libretransform004.obj
 0001:0000144c       nsk_jvmti_lverify          000000018000244c f   libretransform004.obj
 0001:0000153c       nsk_jvmti_resetAgentData   000000018000253c f   libretransform004.obj
 0001:000015bc       nsk_jvmti_setFailStatus    00000001800025bc f   libretransform004.obj
 0001:000015f8       nsk_lcomplain              00000001800025f8 f   libretransform004.obj
 0001:00001618       nsk_ldisplay               0000000180002618 f   libretransform004.obj
 0001:00001638       nsk_ltrace                 0000000180002638 f   libretransform004.obj
 0001:00001658       nsk_lvcomplain             0000000180002658 f   libretransform004.obj
 0001:00001810       nsk_lvdisplay              0000000180002810 f   libretransform004.obj
 0001:0000185c       nsk_lverify                000000018000285c f   libretransform004.obj
 0001:000018b8       nsk_lvtrace                00000001800028b8 f   libretransform004.obj
 0001:00001918       nsk_printf                 0000000180002918 f   libretransform004.obj
 0001:00001940       nsk_vprintf                0000000180002940 f   libretransform004.obj
 0001:000019f4       printf                     00000001800029f4 f i libretransform004.obj
 0001:00001f1c       __raise_securityfailure    0000000180002f1c f   MSVCRT:gs_report.obj
 0001:00001f50       __report_gsfailure         0000000180002f50 f   MSVCRT:gs_report.obj
 0001:00002190       __GSHandlerCheck           0000000180003190 f   MSVCRT:gshandler.obj
 0001:000021b0       __GSHandlerCheckCommon     00000001800031b0 f   MSVCRT:gshandler.obj
 0001:00002220       __security_check_cookie    0000000180003220 f   MSVCRT:amdsecgs.obj
 0001:00002560       _DllMainCRTStartup         0000000180003560 f   MSVCRT:dll_dllmain.obj
 0001:000025a0       __scrt_acquire_startup_lock 00000001800035a0 f   MSVCRT:utility.obj
 0001:000025dc       __scrt_dllmain_after_initialize_c 00000001800035dc f   MSVCRT:utility.obj
 0001:00002610       __scrt_dllmain_before_initialize_c 0000000180003610 f   MSVCRT:utility.obj
 0001:00002628       __scrt_dllmain_crt_thread_attach 0000000180003628 f   MSVCRT:utility.obj
 0001:00002650       __scrt_dllmain_crt_thread_detach 0000000180003650 f   MSVCRT:utility.obj
 0001:00002668       __scrt_dllmain_exception_filter 0000000180003668 f   MSVCRT:utility.obj
 0001:000026c8       __scrt_dllmain_uninitialize_c 00000001800036c8 f   MSVCRT:utility.obj
 0001:000026f8       __scrt_dllmain_uninitialize_critical 00000001800036f8 f   MSVCRT:utility.obj
 0001:0000270c       __scrt_initialize_crt      000000018000370c f   MSVCRT:utility.obj
 0001:00002758       __scrt_initialize_onexit_tables 0000000180003758 f   MSVCRT:utility.obj
 0001:000027e4       __scrt_is_nonwritable_in_current_image 00000001800037e4 f   MSVCRT:utility.obj
 0001:0000287c       __scrt_release_startup_lock 000000018000387c f   MSVCRT:utility.obj
 0001:000028a0       __scrt_uninitialize_crt    00000001800038a0 f   MSVCRT:utility.obj
 0001:000028cc       _onexit                    00000001800038cc f   MSVCRT:utility.obj
 0001:00002908       atexit                     0000000180003908 f   MSVCRT:utility.obj
 0001:00002920       __crt_debugger_hook        0000000180003920 f   MSVCRT:utility_desktop.obj
 0001:00002928       __scrt_fastfail            0000000180003928 f   MSVCRT:utility_desktop.obj
 0001:00002a74       _guard_check_icall_nop     0000000180003a74 f i MSVCRT:guard_support.obj
 0001:00002a78       __security_init_cookie     0000000180003a78 f   MSVCRT:gs_support.obj
 0001:00002b24       DllMain                    0000000180003b24 f   MSVCRT:dll_dllmain_stub.obj
 0001:00002b48       ?__scrt_initialize_type_info@@YAXXZ 0000000180003b48 f   MSVCRT:tncleanup.obj
 0001:00002b58       ?__scrt_uninitialize_type_info@@YAXXZ 0000000180003b58 f   MSVCRT:tncleanup.obj
 0001:00002b64       __local_stdio_scanf_options 0000000180003b64 f i MSVCRT:default_local_stdio_options.obj
 0001:00002b6c       __scrt_initialize_default_local_stdio_options 0000000180003b6c f   MSVCRT:default_local_stdio_options.obj
 0001:00002b88       __scrt_get_dyn_tls_init_callback 0000000180003b88 f   MSVCRT:dyn_tls_init.obj
 0001:00002b90       _RTC_Initialize            0000000180003b90 f   MSVCRT:initsect.obj
 0001:00002bcc       _RTC_Terminate             0000000180003bcc f   MSVCRT:initsect.obj
 0001:00002c08       __isa_available_init       0000000180003c08 f   MSVCRT:cpu_disp.obj
 0001:00002db4       _get_startup_argv_mode     0000000180003db4 f   MSVCRT:argv_mode.obj
 0001:00002dbc       __scrt_is_ucrt_dll_in_use  0000000180003dbc f   MSVCRT:ucrt_detection.obj
 0001:00002dd0       memcpy                     0000000180003dd0 f   vcruntime:VCRUNTIME140.dll
 0001:00002dd6       memset                     0000000180003dd6 f   vcruntime:VCRUNTIME140.dll
 0001:00002ddc       strchr                     0000000180003ddc f   vcruntime:VCRUNTIME140.dll
 0001:00002de2       __C_specific_handler       0000000180003de2 f   vcruntime:VCRUNTIME140.dll
 0001:00002de8       __std_type_info_destroy_list 0000000180003de8 f   vcruntime:VCRUNTIME140.dll
 0001:00002dee       strlen                     0000000180003dee f   ucrt:api-ms-win-crt-string-l1-1-0.dll
 0001:00002df4       _initterm                  0000000180003df4 f   ucrt:api-ms-win-crt-runtime-l1-1-0.dll
 0001:00002dfa       _initterm_e                0000000180003dfa f   ucrt:api-ms-win-crt-runtime-l1-1-0.dll
 0001:00002e00       _seh_filter_dll            0000000180003e00 f   ucrt:api-ms-win-crt-runtime-l1-1-0.dll
 0001:00002e06       _configure_narrow_argv     0000000180003e06 f   ucrt:api-ms-win-crt-runtime-l1-1-0.dll
 0001:00002e0c       _initialize_narrow_environment 0000000180003e0c f   ucrt:api-ms-win-crt-runtime-l1-1-0.dll
 0001:00002e12       _initialize_onexit_table   0000000180003e12 f   ucrt:api-ms-win-crt-runtime-l1-1-0.dll
 0001:00002e18       _register_onexit_function  0000000180003e18 f   ucrt:api-ms-win-crt-runtime-l1-1-0.dll
 0001:00002e1e       _execute_onexit_table      0000000180003e1e f   ucrt:api-ms-win-crt-runtime-l1-1-0.dll
 0001:00002e24       _crt_atexit                0000000180003e24 f   ucrt:api-ms-win-crt-runtime-l1-1-0.dll
 0001:00002e2a       _cexit                     0000000180003e2a f   ucrt:api-ms-win-crt-runtime-l1-1-0.dll
 0001:00002e30       __acrt_initialize          0000000180003e30 f   MSVCRT:ucrt_stubs.obj
 0001:00002e30       __acrt_thread_attach       0000000180003e30 f   MSVCRT:ucrt_stubs.obj
 0001:00002e30       __acrt_thread_detach       0000000180003e30 f   MSVCRT:ucrt_stubs.obj
 0001:00002e30       __acrt_uninitialize        0000000180003e30 f   MSVCRT:ucrt_stubs.obj
 0001:00002e30       __acrt_uninitialize_critical 0000000180003e30 f   MSVCRT:ucrt_stubs.obj
 0001:00002e30       __scrt_stub_for_acrt_initialize 0000000180003e30 f   MSVCRT:ucrt_stubs.obj
 0001:00002e30       __scrt_stub_for_acrt_thread_attach 0000000180003e30 f   MSVCRT:ucrt_stubs.obj
 0001:00002e30       __scrt_stub_for_acrt_thread_detach 0000000180003e30 f   MSVCRT:ucrt_stubs.obj
 0001:00002e30       __scrt_stub_for_acrt_uninitialize 0000000180003e30 f   MSVCRT:ucrt_stubs.obj
 0001:00002e30       __scrt_stub_for_acrt_uninitialize_critical 0000000180003e30 f   MSVCRT:ucrt_stubs.obj
 0001:00002e30       __vcrt_initialize          0000000180003e30 f   MSVCRT:ucrt_stubs.obj
 0001:00002e30       __vcrt_thread_attach       0000000180003e30 f   MSVCRT:ucrt_stubs.obj
 0001:00002e30       __vcrt_thread_detach       0000000180003e30 f   MSVCRT:ucrt_stubs.obj
 0001:00002e30       __vcrt_uninitialize        0000000180003e30 f   MSVCRT:ucrt_stubs.obj
 0001:00002e30       __vcrt_uninitialize_critical 0000000180003e30 f   MSVCRT:ucrt_stubs.obj
 0001:00002e34       __scrt_stub_for_is_c_termination_complete 0000000180003e34 f   MSVCRT:ucrt_stubs.obj
 0001:00002e34       _is_c_termination_complete 0000000180003e34 f   MSVCRT:ucrt_stubs.obj
 0001:00002e50       _guard_dispatch_icall_nop  0000000180003e50 f   MSVCRT:guard_dispatch.obj
 0001:00002e70       _guard_xfg_dispatch_icall_nop 0000000180003e70 f   MSVCRT:guard_xfg_dispatch.obj
 0002:00000000       __imp_RtlCaptureContext    0000000180004000     kernel32:KERNEL32.dll
 0002:00000008       __imp_RtlLookupFunctionEntry 0000000180004008     kernel32:KERNEL32.dll
 0002:00000010       __imp_RtlVirtualUnwind     0000000180004010     kernel32:KERNEL32.dll
 0002:00000018       __imp_UnhandledExceptionFilter 0000000180004018     kernel32:KERNEL32.dll
 0002:00000020       __imp_SetUnhandledExceptionFilter 0000000180004020     kernel32:KERNEL32.dll
 0002:00000028       __imp_GetCurrentProcess    0000000180004028     kernel32:KERNEL32.dll
 0002:00000030       __imp_TerminateProcess     0000000180004030     kernel32:KERNEL32.dll
 0002:00000038       __imp_IsProcessorFeaturePresent 0000000180004038     kernel32:KERNEL32.dll
 0002:00000040       __imp_CloseHandle          0000000180004040     kernel32:KERNEL32.dll
 0002:00000048       __imp_InitializeCriticalSectionAndSpinCount 0000000180004048     kernel32:KERNEL32.dll
 0002:00000050       __imp_DeleteCriticalSection 0000000180004050     kernel32:KERNEL32.dll
 0002:00000058       __imp_CreateEventW         0000000180004058     kernel32:KERNEL32.dll
 0002:00000060       __imp_GetModuleHandleW     0000000180004060     kernel32:KERNEL32.dll
 0002:00000068       __imp_GetProcAddress       0000000180004068     kernel32:KERNEL32.dll
 0002:00000070       __imp_IsDebuggerPresent    0000000180004070     kernel32:KERNEL32.dll
 0002:00000078       __imp_QueryPerformanceCounter 0000000180004078     kernel32:KERNEL32.dll
 0002:00000080       __imp_GetCurrentProcessId  0000000180004080     kernel32:KERNEL32.dll
 0002:00000088       __imp_GetCurrentThreadId   0000000180004088     kernel32:KERNEL32.dll
 0002:00000090       __imp_GetSystemTimeAsFileTime 0000000180004090     kernel32:KERNEL32.dll
 0002:00000098       __imp_DisableThreadLibraryCalls 0000000180004098     kernel32:KERNEL32.dll
 0002:000000a0       __imp_InitializeSListHead  00000001800040a0     kernel32:KERNEL32.dll
 0002:000000a8       \177KERNEL32_NULL_THUNK_DATA 00000001800040a8     kernel32:KERNEL32.dll
 0002:000000b0       __imp_memcpy               00000001800040b0     vcruntime:VCRUNTIME140.dll
 0002:000000b8       __imp_memset               00000001800040b8     vcruntime:VCRUNTIME140.dll
 0002:000000c0       __imp_strchr               00000001800040c0     vcruntime:VCRUNTIME140.dll
 0002:000000c8       __imp___C_specific_handler 00000001800040c8     vcruntime:VCRUNTIME140.dll
 0002:000000d0       __imp___std_type_info_destroy_list 00000001800040d0     vcruntime:VCRUNTIME140.dll
 0002:000000d8       \177VCRUNTIME140_NULL_THUNK_DATA 00000001800040d8     vcruntime:VCRUNTIME140.dll
 0002:000000e0       __imp__errno               00000001800040e0     ucrt:api-ms-win-crt-runtime-l1-1-0.dll
 0002:000000e8       __imp_exit                 00000001800040e8     ucrt:api-ms-win-crt-runtime-l1-1-0.dll
 0002:000000f0       __imp__cexit               00000001800040f0     ucrt:api-ms-win-crt-runtime-l1-1-0.dll
 0002:000000f8       __imp__crt_atexit          00000001800040f8     ucrt:api-ms-win-crt-runtime-l1-1-0.dll
 0002:00000100       __imp__execute_onexit_table 0000000180004100     ucrt:api-ms-win-crt-runtime-l1-1-0.dll
 0002:00000108       __imp__register_onexit_function 0000000180004108     ucrt:api-ms-win-crt-runtime-l1-1-0.dll
 0002:00000110       __imp__initialize_onexit_table 0000000180004110     ucrt:api-ms-win-crt-runtime-l1-1-0.dll
 0002:00000118       __imp__initialize_narrow_environment 0000000180004118     ucrt:api-ms-win-crt-runtime-l1-1-0.dll
 0002:00000120       __imp__configure_narrow_argv 0000000180004120     ucrt:api-ms-win-crt-runtime-l1-1-0.dll
 0002:00000128       __imp__seh_filter_dll      0000000180004128     ucrt:api-ms-win-crt-runtime-l1-1-0.dll
 0002:00000130       __imp__initterm_e          0000000180004130     ucrt:api-ms-win-crt-runtime-l1-1-0.dll
 0002:00000138       __imp__initterm            0000000180004138     ucrt:api-ms-win-crt-runtime-l1-1-0.dll
 0002:00000140       \177api-ms-win-crt-runtime-l1-1-0_NULL_THUNK_DATA 0000000180004140     ucrt:api-ms-win-crt-runtime-l1-1-0.dll
 0002:00000148       __imp___acrt_iob_func      0000000180004148     ucrt:api-ms-win-crt-stdio-l1-1-0.dll
 0002:00000150       __imp_fflush               0000000180004150     ucrt:api-ms-win-crt-stdio-l1-1-0.dll
 0002:00000158       __imp___stdio_common_vsprintf 0000000180004158     ucrt:api-ms-win-crt-stdio-l1-1-0.dll
 0002:00000160       __imp___stdio_common_vfprintf 0000000180004160     ucrt:api-ms-win-crt-stdio-l1-1-0.dll
 0002:00000168       \177api-ms-win-crt-stdio-l1-1-0_NULL_THUNK_DATA 0000000180004168     ucrt:api-ms-win-crt-stdio-l1-1-0.dll
 0002:00000170       __imp__strdup              0000000180004170     ucrt:api-ms-win-crt-string-l1-1-0.dll
 0002:00000170       __imp_strdup               0000000180004170     ucrt:api-ms-win-crt-string-l1-1-0.dll
 0002:00000178       __imp_strlen               0000000180004178     ucrt:api-ms-win-crt-string-l1-1-0.dll
 0002:00000180       __imp_strncpy              0000000180004180     ucrt:api-ms-win-crt-string-l1-1-0.dll
 0002:00000188       \177api-ms-win-crt-string-l1-1-0_NULL_THUNK_DATA 0000000180004188     ucrt:api-ms-win-crt-string-l1-1-0.dll
 0002:00000190       __guard_check_icall_fptr   0000000180004190     MSVCRT:guard_support.obj
 0002:00000198       __guard_xfg_check_icall_fptr 0000000180004198     MSVCRT:guard_support.obj
 0002:000001a0       __guard_dispatch_icall_fptr 00000001800041a0     MSVCRT:guard_support.obj
 0002:000001a8       __guard_xfg_dispatch_icall_fptr 00000001800041a8     MSVCRT:guard_support.obj
 0002:000001b0       __guard_xfg_table_dispatch_icall_fptr 00000001800041b0     MSVCRT:guard_support.obj
 0002:000001b8       __castguard_check_failure_os_handled_fptr 00000001800041b8     MSVCRT:guard_support.obj
 0002:000001c0       __guard_memcpy_fptr        00000001800041c0     vcruntime:softmemtag.obj
 0002:000001c8       __xc_a                     00000001800041c8     MSVCRT:initializers.obj
 0002:000001d0       __xc_z                     00000001800041d0     MSVCRT:initializers.obj
 0002:000001d8       __xi_a                     00000001800041d8     MSVCRT:initializers.obj
 0002:000001e8       __xi_z                     00000001800041e8     MSVCRT:initializers.obj
 0002:000001f0       __xl_a                     00000001800041f0     MSVCRT:tlssup.obj
 0002:000001f8       __xl_z                     00000001800041f8     MSVCRT:tlssup.obj
 0002:00000200       __xp_a                     0000000180004200     MSVCRT:initializers.obj
 0002:00000208       __xp_z                     0000000180004208     MSVCRT:initializers.obj
 0002:00000210       __xt_a                     0000000180004210     MSVCRT:initializers.obj
 0002:00000218       __xt_z                     0000000180004218     MSVCRT:initializers.obj
 0002:00000220       g_refKindStr               0000000180004220     libretransform004.obj
 0002:000003d0       ??_C@_09BPLDFGCI@unknown_0@ 00000001800043d0     libretransform004.obj
 0002:000003e0       ??_C@_0BL@FPNMECJD@JVMTI_HEAP_REFERENCE_CLASS@ 00000001800043e0     libretransform004.obj
 0002:00000400       ??_C@_0BL@FKGKKLNM@JVMTI_HEAP_REFERENCE_FIELD@ 0000000180004400     libretransform004.obj
 0002:00000420       ??_C@_0CD@CAEHCFJF@JVMTI_HEAP_REFERENCE_ARRAY_ELEM@ 0000000180004420     libretransform004.obj
 0002:00000448       ??_C@_0CC@DNEBMCNK@JVMTI_HEAP_REFERENCE_CLASS_LOAD@ 0000000180004448     libretransform004.obj
 0002:00000470       ??_C@_0BN@CJMIPEBB@JVMTI_HEAP_REFERENCE_SIGNERS@ 0000000180004470     libretransform004.obj
 0002:00000490       ??_C@_0CH@HBOIDPEB@JVMTI_HEAP_REFERENCE_PROTECTION@ 0000000180004490     libretransform004.obj
 0002:000004b8       ??_C@_0BP@MDKGDGKL@JVMTI_HEAP_REFERENCE_INTERFACE@ 00000001800044b8     libretransform004.obj
 0002:000004d8       ??_C@_0CC@JJMIHNJH@JVMTI_HEAP_REFERENCE_STATIC_FIE@ 00000001800044d8     libretransform004.obj
 0002:00000500       ??_C@_0CD@IDHEEGID@JVMTI_HEAP_REFERENCE_CONSTANT_P@ 0000000180004500     libretransform004.obj
 0002:00000528       ??_C@_0CA@EFFCHNG@JVMTI_HEAP_REFERENCE_SUPERCLASS@ 0000000180004528     libretransform004.obj
 0002:00000548       ??_C@_0L@PCDFHGCJ@unknown_11@ 0000000180004548     libretransform004.obj
 0002:00000558       ??_C@_0L@NJBICFOK@unknown_12@ 0000000180004558     libretransform004.obj
 0002:00000568       ??_C@_0L@MAADBEKL@unknown_13@ 0000000180004568     libretransform004.obj
 0002:00000578       ??_C@_0L@IPECICGM@unknown_14@ 0000000180004578     libretransform004.obj
 0002:00000588       ??_C@_0L@JGFJLDCN@unknown_15@ 0000000180004588     libretransform004.obj
 0002:00000598       ??_C@_0L@LNHEOAOO@unknown_16@ 0000000180004598     libretransform004.obj
 0002:000005a8       ??_C@_0L@KEGPNBKP@unknown_17@ 00000001800045a8     libretransform004.obj
 0002:000005b8       ??_C@_0L@CDPHMNGA@unknown_18@ 00000001800045b8     libretransform004.obj
 0002:000005c8       ??_C@_0L@DKOMPMCB@unknown_19@ 00000001800045c8     libretransform004.obj
 0002:000005d8       ??_C@_0L@OJGIPJDB@unknown_20@ 00000001800045d8     libretransform004.obj
 0002:000005e8       ??_C@_0CA@KAOFNDEM@JVMTI_HEAP_REFERENCE_JNI_GLOBAL@ 00000001800045e8     libretransform004.obj
 0002:00000608       ??_C@_0CC@HPFAJBK@JVMTI_HEAP_REFERENCE_SYSTEM_CLA@ 0000000180004608     libretransform004.obj
 0002:00000630       ??_C@_0BN@FDEGFOHC@JVMTI_HEAP_REFERENCE_MONITOR@ 0000000180004630     libretransform004.obj
 0002:00000650       ??_C@_0CB@HKIBCMAJ@JVMTI_HEAP_REFERENCE_STACK_LOCA@ 0000000180004650     libretransform004.obj
 0002:00000678       ??_C@_0BP@EAACMMOE@JVMTI_HEAP_REFERENCE_JNI_LOCAL@ 0000000180004678     libretransform004.obj
 0002:00000698       ??_C@_0BM@IJDEOGOE@JVMTI_HEAP_REFERENCE_THREAD@ 0000000180004698     libretransform004.obj
 0002:000006b8       ??_C@_0BL@EDGPPKC@JVMTI_HEAP_REFERENCE_OTHER@ 00000001800046b8     libretransform004.obj
 0002:000006d4       ??_C@_04BCJPDBDA@Code@     00000001800046d4     libretransform004.obj
 0002:000006e0       ??_C@_0BA@OCLMCFKC@LineNumberTable@ 00000001800046e0     libretransform004.obj
 0002:000006f0       ??_C@_0BD@CPAEPILC@LocalVariableTable@ 00000001800046f0     libretransform004.obj
 0002:00000708       ??_C@_0BH@NMBDNHBD@LocalVariableTypeTable@ 0000000180004708     libretransform004.obj
 0002:00000720       ??_C@_0O@HIHEEDNJ@StackMapTable@ 0000000180004720     libretransform004.obj
 0002:00000730       ??_C@_0L@HCDIAMJG@?9?5?$CFs?0?5?$CFd?3?5@ 0000000180004730     libretransform004.obj
 0002:00000740       ??_C@_0JI@HLPECLFI@?$CD?5?4?4?4?6?$CD?5ERROR?3?5too?5many?5complai@ 0000000180004740     libretransform004.obj
 0002:000007e0       ??_C@_0ED@JNEKCCOB@The?5following?5fake?5exception?5st@ 00000001800047e0     libretransform004.obj
 0002:00000828       ??_C@_0CN@FCNMDFBH@nsk?4share?4Fake_Exception_for_RU@ 0000000180004828     libretransform004.obj
 0002:00000858       ??_C@_08PGFFNAEI@?$CI?$CFs?3?$CFd?$CJ?5@ 0000000180004858     libretransform004.obj
 0002:00000868       ??_C@_0DP@IENMAEGI@s?2test?2hotspot?2jtreg?2vmTestbase@ 0000000180004868     libretransform004.obj
 0002:000008a8       ??_C@_0BL@NDJLFFJB@?7at?5nsk_lvcomplain?$CI?$CFs?3?$CFd?$CJ?6@ 00000001800048a8     libretransform004.obj
 0002:000008c8       ??_C@_0BC@JOOKAFKF@?$CD?5ERROR?3?5?$CFs?0?5?$CFd?3?5@ 00000001800048c8     libretransform004.obj
 0002:000008e0       ??_C@_09KJEAHMEH@?$CD?5ERROR?3?5@ 00000001800048e0     libretransform004.obj
 0002:000008ec       ??_C@_02GPIOPFAK@?$DO?$DO@ 00000001800048ec     libretransform004.obj
 0002:000008f0       ??_C@_02FODMEDOG@?$DM?$DM@ 00000001800048f0     libretransform004.obj
 0002:000008f4       ??_C@_02DJGKEECL@?4?4@     00000001800048f4     libretransform004.obj
 0002:000008f8       ??_C@_0O@CJPGJOAF@?9?5?$CFs?0?5?$CFd?3?5?$CFs?5@ 00000001800048f8     libretransform004.obj
 0002:00000908       ??_C@_0CB@IAKPDOIC@?$CD?5?5?5verified?5assertion?5is?5FALSE@ 0000000180004908     libretransform004.obj
 0002:00000930       ??_C@_0CO@LGONDEPD@stdout?3?5fflush?5failed?5?9?5err?$DN?$CFd?5@ 0000000180004930     libretransform004.obj
 0002:00000960       ??_C@_0CO@KBGKJPBD@stderr?3?5fflush?5failed?5?9?5err?$DN?$CFd?5@ 0000000180004960     libretransform004.obj
 0002:00000990       ??_C@_0BB@JCNMKLLK@JVMTI_ERROR_NONE@ 0000000180004990     libretransform004.obj
 0002:000009a8       ??_C@_0BL@LDIMKLPH@JVMTI_ERROR_INVALID_THREAD@ 00000001800049a8     libretransform004.obj
 0002:000009c8       ??_C@_0CB@PJFPAIKJ@JVMTI_ERROR_INVALID_THREAD_GROU@ 00000001800049c8     libretransform004.obj
 0002:000009f0       ??_C@_0BN@LLMKHMNF@JVMTI_ERROR_INVALID_PRIORITY@ 00000001800049f0     libretransform004.obj
 0002:00000a10       ??_C@_0CB@MBOFKAGB@JVMTI_ERROR_THREAD_NOT_SUSPENDE@ 0000000180004a10     libretransform004.obj
 0002:00000a38       ??_C@_0BN@FABOLPBI@JVMTI_ERROR_THREAD_SUSPENDED@ 0000000180004a38     libretransform004.obj
 0002:00000a58       ??_C@_0BN@FDGNOBJM@JVMTI_ERROR_THREAD_NOT_ALIVE@ 0000000180004a58     libretransform004.obj
 0002:00000a78       ??_C@_0BL@GOBIFKNJ@JVMTI_ERROR_INVALID_OBJECT@ 0000000180004a78     libretransform004.obj
 0002:00000a98       ??_C@_0BK@FCMAJPPC@JVMTI_ERROR_INVALID_CLASS@ 0000000180004a98     libretransform004.obj
 0002:00000ab8       ??_C@_0BP@IKLLBKEB@JVMTI_ERROR_CLASS_NOT_PREPARED@ 0000000180004ab8     libretransform004.obj
 0002:00000ad8       ??_C@_0BN@KLPPLKG@JVMTI_ERROR_INVALID_METHODID@ 0000000180004ad8     libretransform004.obj
 0002:00000af8       ??_C@_0BN@BCEKOKND@JVMTI_ERROR_INVALID_LOCATION@ 0000000180004af8     libretransform004.obj
 0002:00000b18       ??_C@_0BM@DFDGPME@JVMTI_ERROR_INVALID_FIELDID@ 0000000180004b18     libretransform004.obj
 0002:00000b38       ??_C@_0BL@NELIEPEC@JVMTI_ERROR_NO_MORE_FRAMES@ 0000000180004b38     libretransform004.obj
 0002:00000b58       ??_C@_0BJ@BDBECFDM@JVMTI_ERROR_OPAQUE_FRAME@ 0000000180004b58     libretransform004.obj
 0002:00000b78       ??_C@_0BK@MIIFNLOB@JVMTI_ERROR_TYPE_MISMATCH@ 0000000180004b78     libretransform004.obj
 0002:00000b98       ??_C@_0BJ@HPCAOILC@JVMTI_ERROR_INVALID_SLOT@ 0000000180004b98     libretransform004.obj
 0002:00000bb8       ??_C@_0BG@CHILOPNI@JVMTI_ERROR_DUPLICATE@ 0000000180004bb8     libretransform004.obj
 0002:00000bd0       ??_C@_0BG@DIEMLHKM@JVMTI_ERROR_NOT_FOUND@ 0000000180004bd0     libretransform004.obj
 0002:00000be8       ??_C@_0BM@NHMCKHOB@JVMTI_ERROR_INVALID_MONITOR@ 0000000180004be8     libretransform004.obj
 0002:00000c08       ??_C@_0BO@PPEDAJGL@JVMTI_ERROR_NOT_MONITOR_OWNER@ 0000000180004c08     libretransform004.obj
 0002:00000c28       ??_C@_0BG@FCAIPEID@JVMTI_ERROR_INTERRUPT@ 0000000180004c28     libretransform004.obj
 0002:00000c40       ??_C@_0CB@EGDBNKOI@JVMTI_ERROR_INVALID_CLASS_FORMA@ 0000000180004c40     libretransform004.obj
 0002:00000c68       ??_C@_0CG@DGKOGIAL@JVMTI_ERROR_CIRCULAR_CLASS_DEFI@ 0000000180004c68     libretransform004.obj
 0002:00000c90       ??_C@_0BP@ICEALPKC@JVMTI_ERROR_FAILS_VERIFICATION@ 0000000180004c90     libretransform004.obj
 0002:00000cb0       ??_C@_0DC@JDACLMIO@JVMTI_ERROR_UNSUPPORTED_REDEFIN@ 0000000180004cb0     libretransform004.obj
 0002:00000ce8       ??_C@_0DE@GKDKNOMJ@JVMTI_ERROR_UNSUPPORTED_REDEFIN@ 0000000180004ce8     libretransform004.obj
 0002:00000d20       ??_C@_0BO@LAFKIOG@JVMTI_ERROR_INVALID_TYPESTATE@ 0000000180004d20     libretransform004.obj
 0002:00000d40       ??_C@_0DH@INDGCLLB@JVMTI_ERROR_UNSUPPORTED_REDEFIN@ 0000000180004d40     libretransform004.obj
 0002:00000d78       ??_C@_0DE@NHEOMMGI@JVMTI_ERROR_UNSUPPORTED_REDEFIN@ 0000000180004d78     libretransform004.obj
 0002:00000db0       ??_C@_0CA@EKPNJOEP@JVMTI_ERROR_UNSUPPORTED_VERSION@ 0000000180004db0     libretransform004.obj
 0002:00000dd0       ??_C@_0BN@OFFMAHHL@JVMTI_ERROR_NAMES_DONT_MATCH@ 0000000180004dd0     libretransform004.obj
 0002:00000df0       ??_C@_0DN@HHBBLAKE@JVMTI_ERROR_UNSUPPORTED_REDEFIN@ 0000000180004df0     libretransform004.obj
 0002:00000e30       ??_C@_0DO@HMBGBGNA@JVMTI_ERROR_UNSUPPORTED_REDEFIN@ 0000000180004e30     libretransform004.obj
 0002:00000e70       ??_C@_0BP@PBECGKHJ@JVMTI_ERROR_UNMODIFIABLE_CLASS@ 0000000180004e70     libretransform004.obj
 0002:00000e90       ??_C@_0BK@CANILEHF@JVMTI_ERROR_NOT_AVAILABLE@ 0000000180004e90     libretransform004.obj
 0002:00000eb0       ??_C@_0CE@INJKMEFK@JVMTI_ERROR_MUST_POSSESS_CAPABI@ 0000000180004eb0     libretransform004.obj
 0002:00000ed8       ??_C@_0BJ@LBFPFPDM@JVMTI_ERROR_NULL_POINTER@ 0000000180004ed8     libretransform004.obj
 0002:00000ef8       ??_C@_0BP@CHJPNNEM@JVMTI_ERROR_ABSENT_INFORMATION@ 0000000180004ef8     libretransform004.obj
 0002:00000f18       ??_C@_0BP@OMFMNLC@JVMTI_ERROR_INVALID_EVENT_TYPE@ 0000000180004f18     libretransform004.obj
 0002:00000f38       ??_C@_0BN@BIBNPHHO@JVMTI_ERROR_ILLEGAL_ARGUMENT@ 0000000180004f38     libretransform004.obj
 0002:00000f58       ??_C@_0BK@KKNDHDCE@JVMTI_ERROR_NATIVE_METHOD@ 0000000180004f58     libretransform004.obj
 0002:00000f78       ??_C@_0BK@PMKCFHAE@JVMTI_ERROR_OUT_OF_MEMORY@ 0000000180004f78     libretransform004.obj
 0002:00000f98       ??_C@_0BK@NNJBDMNB@JVMTI_ERROR_ACCESS_DENIED@ 0000000180004f98     libretransform004.obj
 0002:00000fb8       ??_C@_0BI@GHECLMNC@JVMTI_ERROR_WRONG_PHASE@ 0000000180004fb8     libretransform004.obj
 0002:00000fd0       ??_C@_0BF@OLIHJOII@JVMTI_ERROR_INTERNAL@ 0000000180004fd0     libretransform004.obj
 0002:00000fe8       ??_C@_0BO@EOHGKJHI@JVMTI_ERROR_UNATTACHED_THREAD@ 0000000180004fe8     libretransform004.obj
 0002:00001008       ??_C@_0CA@LKHFDACL@JVMTI_ERROR_INVALID_ENVIRONMENT@ 0000000180005008     libretransform004.obj
 0002:00001028       ??_C@_0BA@MMFHLOKK@?$DMunknown?5error?$DO@ 0000000180005028     libretransform004.obj
 0002:00001038       ??_C@_0CF@CBHOKDB@throwable?5?$DN?5jni?9?$DOExceptionOccur@ 0000000180005038     libretransform004.obj
 0002:00001060       ??_C@_03OFAPEBGM@?$CFs?6@  0000000180005060     libretransform004.obj
 0002:00001068       ??_C@_0DM@LPIGEGNJ@s?2test?2hotspot?2jtreg?2vmTestbase@ 0000000180005068     libretransform004.obj
 0002:000010a8       ??_C@_0CC@NFCNPEPK@Exception?5in?5JNI?5call?5?$CIcleared?$CJ@ 00000001800050a8     libretransform004.obj
 0002:000010d0       ??_C@_0BJ@IBAKFIKF@jni?9?$DOExceptionDescribe?$CI?$CJ@ 00000001800050d0     libretransform004.obj
 0002:000010f0       ??_C@_0BG@GGKALKMH@jni?9?$DOExceptionClear?$CI?$CJ@ 00000001800050f0     libretransform004.obj
 0002:00001108       ??_C@_0CF@JMGFGJLJ@?$CD?5?5?5verified?5JNI?5assertion?5is?5F@ 0000000180005108     libretransform004.obj
 0002:00001130       ??_C@_0CB@MLNJNCLJ@?5?5jvmti?5error?3?5code?$DN?$CFd?0?5name?$DN?$CFs@ 0000000180005130     libretransform004.obj
 0002:00001158       ??_C@_0CD@OHBGDKMK@?$CD?5?5?5jvmti?5error?3?5code?$DN?$CFd?0?5name?$DN@ 0000000180005158     libretransform004.obj
 0002:00001180       ??_C@_0CG@JNNCGPHB@?$CD?5?5?5error?5expected?3?5code?$DN?$CFd?0?5na@ 0000000180005180     libretransform004.obj
 0002:000011b0       ??_C@_0EB@IMGKPCGE@?$CIstr_obj?5?$DN?5jni?9?$DONewStringUTF?$CIco@ 00000001800051b0     libretransform004.obj
 0002:00001200       ??_C@_0EA@HFOGGBCC@s?2test?2hotspot?2jtreg?2vmTestbase@ 0000000180005200     libretransform004.obj
 0002:00001240       ??_C@_05KKCIMGE@error@     0000000180005240     libretransform004.obj
 0002:00001248       ??_C@_0CJ@JACLEAA@Test?5failed?5by?5setFailStatus?$CI?$CJ?4@ 0000000180005248     libretransform004.obj
 0002:00001278       ??_C@_0BD@HGNAOMCP@agent_data_monitor@ 0000000180005278     libretransform004.obj
 0002:00001290       ??_C@_0EB@OGCLGKLN@javaVM?9?$DOGetEnv?$CI?$CIvoid?5?$CK?$CK?$CJ?$CGjvmti_@ 0000000180005290     libretransform004.obj
 0002:000012e0       ??_C@_0EA@PNBCDMOA@s?2test?2hotspot?2jtreg?2vmTestbase@ 00000001800052e0     libretransform004.obj
 0002:00001320       ??_C@_0CI@DDPIFBGM@init_agent_data?$CIjvmti_env?0?5?$CGage@ 0000000180005320     libretransform004.obj
 0002:00001348       ??_C@_0DI@ILAHDLMP@?$CI?$CKagentThreadProc?$CJ?$CIjvmti_env?0?5a@ 0000000180005348     libretransform004.obj
 0002:00001380       ??_C@_0BD@KDBALNLB@JVMTI?5agent?5thread@ 0000000180005380     libretransform004.obj
 0002:00001398       ??_C@_0BB@NOKBFPFO@java?1lang?1Thread@ 0000000180005398     libretransform004.obj
 0002:000013ac       ??_C@_06FALKBLGB@?$DMinit?$DO@ 00000001800053ac     libretransform004.obj
 0002:000013b8       ??_C@_0BG@IKDDPPGD@?$CILjava?1lang?1String?$DL?$CJV@ 00000001800053b8     libretransform004.obj
 0002:000013d0       ??_C@_0EB@IFJBFEKC@?$CIthreadClass?5?$DN?5jni_env?9?$DOFindCla@ 00000001800053d0     libretransform004.obj
 0002:00001420       ??_C@_0GF@FGFIBKKL@?$CIthreadCtor?5?$DN?5jni_env?9?$DOGetMetho@ 0000000180005420     libretransform004.obj
 0002:00001488       ??_C@_0DN@NCPDJLOG@?$CIthreadName?5?$DN?5jni_env?9?$DONewStrin@ 0000000180005488     libretransform004.obj
 0002:000014d0       ??_C@_0FE@PFKODBGC@?$CIthreadObject?5?$DN?5jni_env?9?$DONewObj@ 00000001800054d0     libretransform004.obj
 0002:00001530       ??_C@_0ED@HOBAHHJI@?$CIthreadGlobalRef?5?$DN?5jni_env?9?$DONew@ 0000000180005530     libretransform004.obj
 0002:00001580       ??_C@_0FN@HNJJAHFC@jvmti_env?9?$DORunAgentThread?$CIagent@ 0000000180005580     libretransform004.obj
 0002:000015e0       ??_C@_0EA@MOJDNKDF@Debuggee?5status?5sync?5aborted?5be@ 00000001800055e0     libretransform004.obj
 0002:00001620       ??_C@_0EA@EEOEJAEN@status?5?$DN?5syncDebuggeeStatus?$CIjni@ 0000000180005620     libretransform004.obj
 0002:00001660       ??_C@_0BL@JBCFNBMB@nsk_jvmti_resetAgentData?$CI?$CJ@ 0000000180005660     libretransform004.obj
 0002:00001680       ??_C@_0EL@LPBEELIP@s?2test?2hotspot?2jtreg?2vmTestbase@ 0000000180005680     libretransform004.obj
 0002:000016d0       ??_C@_0CK@JDAMFDMJ@jvmti?9?$DOSetTag?$CIo?0?5tag?$CJ?5?$DN?$DN?5JVMTI_@ 00000001800056d0     libretransform004.obj
 0002:00001700       ??_C@_0CC@DAMNHKNI@Can?8t?5set?5tag?5?$CFli?5for?5object?5?$CFl@ 0000000180005700     libretransform004.obj
 0002:00001728       ??_C@_0DL@HAJPNKEF@jvmti?9?$DOGetObjectHashCode?$CIo?0?5?$CGha@ 0000000180005728     libretransform004.obj
 0002:00001768       ??_C@_0BL@JFPIEOBF@Can?8t?5get?5hash?5object?5?$CFlx?6@ 0000000180005768     libretransform004.obj
 0002:00001788       ??_C@_0BG@DICPHBKN@setTag?3?5?$CF08x?5?$DM?9?5?$CF?53li@ 0000000180005788     libretransform004.obj
 0002:000017a0       ??_C@_0DH@FCEEBDMJ@?$CIs?5?$DN?5jni?9?$DOGetStringUTFChars?$CIsIn@ 00000001800057a0     libretransform004.obj
 0002:000017d8       ??_C@_0BJ@OKKGHDCN@Can?8t?5get?5string?5at?5?$CF?$CDp?6@ 00000001800057d8     libretransform004.obj
 0002:000017f8       ??_C@_0BP@EKFLGGFJ@Can?8t?5get?5string?5at?5?$CF?$CDp?3?5null?6@ 00000001800057f8     libretransform004.obj
 0002:00001818       ??_C@_06ICODBHCL@?5?1?1?5?$CFs@ 0000000180005818     libretransform004.obj
 0002:00001820       ??_C@_0DB@KGFPLEGO@?$CIr?5?$DN?5jvmti?9?$DOGetTag?$CIo?0?5?$CGtag?$CJ?$CJ?5?$DN?$DN@ 0000000180005820     libretransform004.obj
 0002:00001858       ??_C@_0CO@PDAGBCGJ@Can?8t?5GetTag?5for?5object?5?$CFlx?4?5Re@ 0000000180005858     libretransform004.obj
 0002:00001888       ??_C@_0CH@HPEODOHC@TEST_BUG?3?5Max?4?5number?5of?5refs?5r@ 0000000180005888     libretransform004.obj
 0002:000018b0       ??_C@_0DI@PHFCABIM@?$CIr?5?$DN?5jvmti?9?$DOGetTag?$CIfrom?0?5?$CGtagFr@ 00000001800058b0     libretransform004.obj
 0002:000018e8       ??_C@_0DI@MDEGFNKD@TEST_BUG?3?5Can?8t?5GetTag?5for?5obje@ 00000001800058e8     libretransform004.obj
 0002:00001920       ??_C@_0DE@MLELJAHM@?$CIr?5?$DN?5jvmti?9?$DOGetTag?$CIto?0?5?$CGtagTo?$CJ?$CJ@ 0000000180005920     libretransform004.obj
 0002:00001958       ??_C@_0DK@IDDJHKEA@jvmti?9?$DORetransformClasses?$CI1?0?5?$CGc@ 0000000180005958     libretransform004.obj
 0002:000019a0       ??_C@_0FP@BJIINGBN@s?2test?2hotspot?2jtreg?2vmTestbase@ 00000001800059a0     libretransform004.obj
 0002:00001a00       ??_C@_0DA@GMFPINEC@jvmti?9?$DOAllocate?$CIclass_data_len?0@ 0000000180005a00     libretransform004.obj
 0002:00001a30       ??_C@_0DM@OFHPOAIH@?$CIjvmti?5?$DN?5nsk_jvmti_createJVMTIE@ 0000000180005a30     libretransform004.obj
 0002:00001a70       ??_C@_0BO@IAKFILDF@jvmti?9?$DOGetCapabilities?$CI?$CGcaps?$CJ@ 0000000180005a70     libretransform004.obj
 0002:00001a90       ??_C@_0BO@DBKDIPGD@jvmti?9?$DOAddCapabilities?$CI?$CGcaps?$CJ@ 0000000180005a90     libretransform004.obj
 0002:00001ab0       ??_C@_0DI@NJCFGEGC@jvmti?9?$DOSetEventCallbacks?$CI?$CGcallb@ 0000000180005ab0     libretransform004.obj
 0002:00001af0       ??_C@_0FJ@EBLPDPLG@jvmti?9?$DOSetEventNotificationMode@ 0000000180005af0     libretransform004.obj
 0002:00001b60       ??_C@_1EC@JIJBPKFM@?$AAa?$AAp?$AAi?$AA?9?$AAm?$AAs?$AA?9?$AAw?$AAi?$AAn?$AA?9?$AAc?$AAo?$AAr?$AAe@ 0000000180005b60     MSVCRT:thread_safe_statics.obj
 0002:00001ba8       ??_C@_1BK@MGMFAEKH@?$AAk?$AAe?$AAr?$AAn?$AAe?$AAl?$AA3?$AA2?$AA?4?$AAd?$AAl?$AAl@ 0000000180005ba8     MSVCRT:thread_safe_statics.obj
 0002:00001bc8       ??_C@_0BJ@JEBJOJFJ@SleepConditionVariableCS@ 0000000180005bc8     MSVCRT:thread_safe_statics.obj
 0002:00001be8       ??_C@_0BJ@PGPPEPCC@WakeAllConditionVariable@ 0000000180005be8     MSVCRT:thread_safe_statics.obj
 0002:00001c08       _pDefaultRawDllMain        0000000180005c08     MSVCRT:dll_dllmain.obj
 0002:00001c08       _pRawDllMain               0000000180005c08     MSVCRT:dll_dllmain.obj
 0002:00001c10       __xmm@ffffffffffffffffffffffffffffffff 0000000180005c10     MSVCRT:utility.obj
 0002:00001c20       _load_config_used          0000000180005c20     MSVCRT:loadcfg.obj
 0002:00001e00       _tls_used                  0000000180005e00     MSVCRT:tlssup.obj
 0002:00001e28       __volatile_metadata        0000000180005e28     <linker-defined>
 0002:000021f0       __rtc_iaa                  00000001800061f0     MSVCRT:initsect.obj
 0002:000021f8       __rtc_izz                  00000001800061f8     MSVCRT:initsect.obj
 0002:00002200       __rtc_taa                  0000000180006200     MSVCRT:initsect.obj
 0002:00002208       __rtc_tzz                  0000000180006208     MSVCRT:initsect.obj
 0002:00002210       _tls_start                 0000000180006210     MSVCRT:tlssup.obj
 0002:00002214       _Init_thread_epoch         0000000180006214     MSVCRT:thread_safe_statics.obj
 0002:00002218       _tls_end                   0000000180006218     MSVCRT:tlssup.obj
 0002:00002914       __IMPORT_DESCRIPTOR_KERNEL32 0000000180006914     kernel32:KERNEL32.dll
 0002:00002928       __IMPORT_DESCRIPTOR_VCRUNTIME140 0000000180006928     vcruntime:VCRUNTIME140.dll
 0002:0000293c       __IMPORT_DESCRIPTOR_api-ms-win-crt-runtime-l1-1-0 000000018000693c     ucrt:api-ms-win-crt-runtime-l1-1-0.dll
 0002:00002950       __IMPORT_DESCRIPTOR_api-ms-win-crt-stdio-l1-1-0 0000000180006950     ucrt:api-ms-win-crt-stdio-l1-1-0.dll
 0002:00002964       __IMPORT_DESCRIPTOR_api-ms-win-crt-string-l1-1-0 0000000180006964     ucrt:api-ms-win-crt-string-l1-1-0.dll
 0002:00002978       __NULL_IMPORT_DESCRIPTOR   0000000180006978     kernel32:KERNEL32.dll
 0003:00000030       _Init_global_epoch         0000000180007030     MSVCRT:thread_safe_statics.obj
 0003:00000040       __security_cookie          0000000180007040     MSVCRT:gs_cookie.obj
 0003:00000048       __security_cookie_complement 0000000180007048     MSVCRT:gs_cookie.obj
 0003:00000050       __scrt_native_dllmain_reason 0000000180007050     MSVCRT:utility.obj
 0003:00000058       __isa_available            0000000180007058     MSVCRT:cpu_disp.obj
 0003:0000005c       __isa_enabled              000000018000705c     MSVCRT:cpu_disp.obj
 0003:00000060       __memset_fast_string_threshold 0000000180007060     MSVCRT:cpu_disp.obj
 0003:00000068       __memset_nt_threshold      0000000180007068     MSVCRT:cpu_disp.obj
 0003:00000070       __scrt_ucrt_dll_is_in_use  0000000180007070     MSVCRT:ucrt_stubs.obj
 0003:00000080       g_wrongHeapCallbacks       0000000180007080     libretransform004.obj
 0003:00000100       g_szTagInfo                0000000180007100     libretransform004.obj
 0003:00002040       g_tagFlags                 0000000180009040     libretransform004.obj
 0003:00002428       g_refsToVerifyCnt          0000000180009428     libretransform004.obj
 0003:0000242c       g_fakeUserData             000000018000942c     libretransform004.obj
 0003:00002430       g_tagVisitCount            0000000180009430     libretransform004.obj
 0003:000033d0       g_refsToVerify             000000018000a3d0     libretransform004.obj
 0003:0001aad0       g_userDataError            0000000180021ad0     libretransform004.obj
 0003:0001ac70       ?_OptionsStorage@?1??__local_stdio_printf_options@@9@4_KA 0000000180021c70     libretransform004.obj
 0003:0001b238       _tls_index                 0000000180022238     MSVCRT:tlssup.obj
 0003:0001b240       __scrt_current_native_startup_state 0000000180022240     MSVCRT:utility.obj
 0003:0001b248       __scrt_native_startup_lock 0000000180022248     MSVCRT:utility.obj
 0003:0001b288       __scrt_debugger_hook_flag  0000000180022288     MSVCRT:utility_desktop.obj
 0003:0001b290       ?__type_info_root_node@@3U__type_info_node@@A 0000000180022290     MSVCRT:tncleanup.obj
 0003:0001b2a0       ?_OptionsStorage@?1??__local_stdio_scanf_options@@9@4_KA 00000001800222a0     MSVCRT:default_local_stdio_options.obj
 0003:0001b2a8       __favor                    00000001800222a8     MSVCRT:cpu_disp.obj
 0003:0001b2b0       __dyn_tls_init_callback    00000001800222b0     <common>

 entry point at        0001:00002560

 Static symbols

 0000:fffdb000       .debug$S                   0000000180000000     retransform004.exp
 0000:fffdb000       .debug$S                   0000000180000000     vcruntime:VCRUNTIME140.dll
 0000:fffdb000       .debug$S                   0000000180000000     vcruntime:VCRUNTIME140.dll
 0000:fffdb000       .debug$S                   0000000180000000     vcruntime:VCRUNTIME140.dll
 0000:fffdb000       .debug$S                   0000000180000000     vcruntime:VCRUNTIME140.dll
 0000:fffdb000       .debug$S                   0000000180000000     vcruntime:VCRUNTIME140.dll
 0000:fffdb000       .debug$S                   0000000180000000     vcruntime:VCRUNTIME140.dll
 0000:fffdb000       .debug$S                   0000000180000000     vcruntime:VCRUNTIME140.dll
 0000:fffdb000       .debug$S                   0000000180000000     ucrt:api-ms-win-crt-convert-l1-1-0.dll
 0002:ffffc000       .idata$6                   0000000180000000     ucrt:api-ms-win-crt-convert-l1-1-0.dll
 0000:fffdb000       .debug$S                   0000000180000000     ucrt:api-ms-win-crt-heap-l1-1-0.dll
 0000:fffdb000       .debug$S                   0000000180000000     ucrt:api-ms-win-crt-heap-l1-1-0.dll
 0000:fffdb000       .debug$S                   0000000180000000     ucrt:api-ms-win-crt-heap-l1-1-0.dll
 0000:fffdb000       .debug$S                   0000000180000000     ucrt:api-ms-win-crt-heap-l1-1-0.dll
 0002:ffffc000       .idata$6                   0000000180000000     ucrt:api-ms-win-crt-heap-l1-1-0.dll
 0000:fffdb000       .debug$S                   0000000180000000     ucrt:api-ms-win-crt-runtime-l1-1-0.dll
 0000:fffdb000       .debug$S                   0000000180000000     ucrt:api-ms-win-crt-runtime-l1-1-0.dll
 0000:fffdb000       .debug$S                   0000000180000000     ucrt:api-ms-win-crt-runtime-l1-1-0.dll
 0000:fffdb000       .debug$S                   0000000180000000     ucrt:api-ms-win-crt-runtime-l1-1-0.dll
 0000:fffdb000       .debug$S                   0000000180000000     ucrt:api-ms-win-crt-runtime-l1-1-0.dll
 0000:fffdb000       .debug$S                   0000000180000000     ucrt:api-ms-win-crt-runtime-l1-1-0.dll
 0000:fffdb000       .debug$S                   0000000180000000     ucrt:api-ms-win-crt-runtime-l1-1-0.dll
 0000:fffdb000       .debug$S                   0000000180000000     ucrt:api-ms-win-crt-runtime-l1-1-0.dll
 0000:fffdb000       .debug$S                   0000000180000000     ucrt:api-ms-win-crt-runtime-l1-1-0.dll
 0000:fffdb000       .debug$S                   0000000180000000     ucrt:api-ms-win-crt-runtime-l1-1-0.dll
 0000:fffdb000       .debug$S                   0000000180000000     ucrt:api-ms-win-crt-runtime-l1-1-0.dll
 0000:fffdb000       .debug$S                   0000000180000000     ucrt:api-ms-win-crt-runtime-l1-1-0.dll
 0000:fffdb000       .debug$S                   0000000180000000     ucrt:api-ms-win-crt-runtime-l1-1-0.dll
 0000:fffdb000       .debug$S                   0000000180000000     ucrt:api-ms-win-crt-runtime-l1-1-0.dll
 0000:fffdb000       .debug$S                   0000000180000000     ucrt:api-ms-win-crt-runtime-l1-1-0.dll
 0000:fffdb000       .debug$S                   0000000180000000     ucrt:api-ms-win-crt-runtime-l1-1-0.dll
 0000:fffdb000       .debug$S                   0000000180000000     ucrt:api-ms-win-crt-stdio-l1-1-0.dll
 0000:fffdb000       .debug$S                   0000000180000000     ucrt:api-ms-win-crt-stdio-l1-1-0.dll
 0000:fffdb000       .debug$S                   0000000180000000     ucrt:api-ms-win-crt-stdio-l1-1-0.dll
 0000:fffdb000       .debug$S                   0000000180000000     ucrt:api-ms-win-crt-stdio-l1-1-0.dll
 0000:fffdb000       .debug$S                   0000000180000000     ucrt:api-ms-win-crt-stdio-l1-1-0.dll
 0000:fffdb000       .debug$S                   0000000180000000     ucrt:api-ms-win-crt-stdio-l1-1-0.dll
 0000:fffdb000       .debug$S                   0000000180000000     ucrt:api-ms-win-crt-stdio-l1-1-0.dll
 0000:fffdb000       .debug$S                   0000000180000000     ucrt:api-ms-win-crt-stdio-l1-1-0.dll
 0000:fffdb000       .debug$S                   0000000180000000     ucrt:api-ms-win-crt-stdio-l1-1-0.dll
 0000:fffdb000       .debug$S                   0000000180000000     ucrt:api-ms-win-crt-stdio-l1-1-0.dll
 0000:fffdb000       .debug$S                   0000000180000000     ucrt:api-ms-win-crt-string-l1-1-0.dll
 0000:fffdb000       .debug$S                   0000000180000000     ucrt:api-ms-win-crt-string-l1-1-0.dll
 0000:fffdb000       .debug$S                   0000000180000000     ucrt:api-ms-win-crt-string-l1-1-0.dll
 0000:fffdb000       .debug$S                   0000000180000000     ucrt:api-ms-win-crt-string-l1-1-0.dll
 0000:fffdb000       .debug$S                   0000000180000000     ucrt:api-ms-win-crt-string-l1-1-0.dll
 0000:fffdb000       .debug$S                   0000000180000000     ucrt:api-ms-win-crt-string-l1-1-0.dll
 0000:fffdb000       .debug$S                   0000000180000000     ucrt:api-ms-win-crt-string-l1-1-0.dll
 0000:fffdb000       .debug$S                   0000000180000000     ucrt:api-ms-win-crt-string-l1-1-0.dll
 0000:fffdb000       .debug$S                   0000000180000000     kernel32:KERNEL32.dll
 0000:fffdb000       .debug$S                   0000000180000000     kernel32:KERNEL32.dll
 0000:fffdb000       .debug$S                   0000000180000000     kernel32:KERNEL32.dll
 0000:fffdb000       .debug$S                   0000000180000000     kernel32:KERNEL32.dll
 0000:fffdb000       .debug$S                   0000000180000000     kernel32:KERNEL32.dll
 0000:fffdb000       .debug$S                   0000000180000000     kernel32:KERNEL32.dll
 0000:fffdb000       .debug$S                   0000000180000000     kernel32:KERNEL32.dll
 0000:fffdb000       .debug$S                   0000000180000000     kernel32:KERNEL32.dll
 0000:fffdb000       .debug$S                   0000000180000000     kernel32:KERNEL32.dll
 0000:fffdb000       .debug$S                   0000000180000000     kernel32:KERNEL32.dll
 0000:fffdb000       .debug$S                   0000000180000000     kernel32:KERNEL32.dll
 0000:fffdb000       .debug$S                   0000000180000000     kernel32:KERNEL32.dll
 0000:fffdb000       .debug$S                   0000000180000000     kernel32:KERNEL32.dll
 0000:fffdb000       .debug$S                   0000000180000000     kernel32:KERNEL32.dll
 0000:fffdb000       .debug$S                   0000000180000000     kernel32:KERNEL32.dll
 0000:fffdb000       .debug$S                   0000000180000000     kernel32:KERNEL32.dll
 0000:fffdb000       .debug$S                   0000000180000000     kernel32:KERNEL32.dll
 0000:fffdb000       .debug$S                   0000000180000000     kernel32:KERNEL32.dll
 0000:fffdb000       .debug$S                   0000000180000000     kernel32:KERNEL32.dll
 0000:fffdb000       .debug$S                   0000000180000000     kernel32:KERNEL32.dll
 0000:fffdb000       .debug$S                   0000000180000000     kernel32:KERNEL32.dll
 0000:fffdb000       .debug$S                   0000000180000000     kernel32:KERNEL32.dll
 0000:fffdb000       .debug$S                   0000000180000000     kernel32:KERNEL32.dll
 0000:fffdb000       .debug$S                   0000000180000000     kernel32:KERNEL32.dll
 0000:fffdb000       .debug$S                   0000000180000000     kernel32:KERNEL32.dll
 0000:fffdb000       .debug$S                   0000000180000000     kernel32:KERNEL32.dll
 0000:fffdb000       .debug$S                   0000000180000000     kernel32:KERNEL32.dll
 0000:fffdb000       .debug$S                   0000000180000000     kernel32:KERNEL32.dll
 0001:00000748       ClassFileLoadHook          0000000180001748 f   libretransform004.obj
 0001:0000104c       addRefToVerify             000000018000204c f   libretransform004.obj
 0001:000010b8       agentThreadWrapper         00000001800020b8 f   libretransform004.obj
 0001:000012a8       file_basename              00000001800022a8 f   libretransform004.obj
 0001:00001a44       startAgentThreadWrapper    0000000180002a44 f   libretransform004.obj
 0001:00001d84       syncDebuggeeStatus         0000000180002d84 f   libretransform004.obj
 0001:00002024       capture_previous_context   0000000180003024 f   MSVCRT:gs_report.obj
 0001:00002098       ?__scrt_initialize_thread_safe_statics@@YAHXZ 0000000180003098 f   MSVCRT:thread_safe_statics.obj
 0001:00002168       ?__scrt_uninitialize_thread_safe_statics@@YAXXZ 0000000180003168 f   MSVCRT:thread_safe_statics.obj
 0001:00002210       $$000000                   0000000180003210     MSVCRT:amdsecgs.obj
 0001:00002240       ?dllmain_crt_dispatch@@YAHQEAUHINSTANCE__@@KQEAX@Z 0000000180003240 f   MSVCRT:dll_dllmain.obj
 0001:00002290       ?dllmain_crt_process_attach@@YAHQEAUHINSTANCE__@@QEAX@Z 0000000180003290 f   MSVCRT:dll_dllmain.obj
 0001:000023a8       ?dllmain_crt_process_detach@@YAH_N@Z 00000001800033a8 f   MSVCRT:dll_dllmain.obj
 0001:0000242c       ?dllmain_dispatch@@YAHQEAUHINSTANCE__@@KQEAX@Z 000000018000342c f   MSVCRT:dll_dllmain.obj
 0001:00002e40       $$000000                   0000000180003e40     MSVCRT:guard_dispatch.obj
 0001:00002e60       $$000000                   0000000180003e60     MSVCRT:guard_xfg_dispatch.obj
 0001:00002e76       ?fin$0@?0??dllmain_crt_process_attach@@YAHQEAUHINSTANCE__@@QEAX@Z@4HA 0000000180003e76 f   MSVCRT:dll_dllmain.obj
 0001:00002e8d       ?fin$0@?0??dllmain_crt_process_detach@@YAH_N@Z@4HA 0000000180003e8d f   MSVCRT:dll_dllmain.obj
 0001:00002ea6       ?fin$1@?0??dllmain_crt_process_detach@@YAH_N@Z@4HA 0000000180003ea6 f   MSVCRT:dll_dllmain.obj
 0001:00002eba       ?filt$0@?0??dllmain_dispatch@@YAHQEAUHINSTANCE__@@KQEAX@Z@4HA 0000000180003eba f   MSVCRT:dll_dllmain.obj
 0001:00002ef0       __scrt_is_nonwritable_in_current_image$filt$0 0000000180003ef0 f   MSVCRT:utility.obj
 0002:000001e0       ?__scrt_initialize_tss_var@@3P6AHXZEA 00000001800041e0     MSVCRT:thread_safe_statics.obj
 0002:00000300       ?opcLengths@@3QBEB         0000000180004300     libretransform004.obj
 0002:00001b50       GS_ExceptionPointers       0000000180005b50     MSVCRT:gs_report.obj
 0002:00002220       $unwind$fprintf            0000000180006220     libretransform004.obj
 0002:0000222c       $unwind$printf             000000018000622c     libretransform004.obj
 0002:00002238       $unwind$?NewObject@JNIEnv_@@QEAAPEAV_jobject@@PEAV_jclass@@PEAU_jmethodID@@ZZ 0000000180006238     libretransform004.obj
 0002:00002238       $unwind$nsk_lcomplain      0000000180006238     libretransform004.obj
 0002:00002238       $unwind$nsk_ldisplay       0000000180006238     libretransform004.obj
 0002:00002240       $unwind$nsk_lvdisplay      0000000180006240     libretransform004.obj
 0002:00002240       $unwind$_RTC_Initialize    0000000180006240     MSVCRT:initsect.obj
 0002:00002240       $unwind$_RTC_Terminate     0000000180006240     MSVCRT:initsect.obj
 0002:00002240       $unwind$?__scrt_initialize_thread_safe_statics@@YAHXZ 0000000180006240     MSVCRT:thread_safe_statics.obj
 0002:0000224c       $unwind$nsk_lvcomplain     000000018000624c     libretransform004.obj
 0002:00002264       $unwind$nsk_ltrace         0000000180006264     libretransform004.obj
 0002:00002264       $unwind$__report_gsfailure 0000000180006264     MSVCRT:gs_report.obj
 0002:0000226c       $unwind$nsk_lvtrace        000000018000626c     libretransform004.obj
 0002:0000226c       $unwind$__raise_securityfailure 000000018000626c     MSVCRT:gs_report.obj
 0002:0000226c       $unwind$__scrt_initialize_crt 000000018000626c     MSVCRT:utility.obj
 0002:0000226c       $unwind$__scrt_initialize_onexit_tables 000000018000626c     MSVCRT:utility.obj
 0002:0000226c       $unwind$__scrt_release_startup_lock 000000018000626c     MSVCRT:utility.obj
 0002:0000226c       $unwind$__scrt_uninitialize_crt 000000018000626c     MSVCRT:utility.obj
 0002:0000226c       $unwind$_onexit            000000018000626c     MSVCRT:utility.obj
 0002:00002274       $unwind$nsk_lverify        0000000180006274     libretransform004.obj
 0002:00002284       $unwind$nsk_vprintf        0000000180006284     libretransform004.obj
 0002:00002294       $unwind$nsk_printf         0000000180006294     libretransform004.obj
 0002:0000229c       $unwind$?nsk_jni_lverify@@YAHHPEAUJNIEnv_@@HQEBDH1ZZ 000000018000629c     libretransform004.obj
 0002:000022b0       $unwind$?nsk_jni_check_exception@@YAHPEAUJNIEnv_@@QEBDH@Z 00000001800062b0     libretransform004.obj
 0002:000022cc       $unwind$nsk_jvmti_createJVMTIEnv 00000001800062cc     libretransform004.obj
 0002:000022e0       $unwind$Java_nsk_jvmti_unit_FollowReferences_FollowRefObjects_resetTags 00000001800062e0     libretransform004.obj
 0002:000022e0       $unwind$addRefToVerify     00000001800062e0     libretransform004.obj
 0002:000022e0       $unwind$nsk_jvmti_resetAgentData 00000001800062e0     libretransform004.obj
 0002:000022e0       $unwind$nsk_jvmti_setFailStatus 00000001800062e0     libretransform004.obj
 0002:000022e0       $unwind$__scrt_initialize_default_local_stdio_options 00000001800062e0     MSVCRT:default_local_stdio_options.obj
 0002:000022e0       $unwind$?dllmain_crt_dispatch@@YAHQEAUHINSTANCE__@@KQEAX@Z 00000001800062e0     MSVCRT:dll_dllmain.obj
 0002:000022e0       $unwind$DllMain            00000001800062e0     MSVCRT:dll_dllmain_stub.obj
 0002:000022e0       $unwind$__GSHandlerCheck   00000001800062e0     MSVCRT:gshandler.obj
 0002:000022e0       $unwind$?__scrt_uninitialize_thread_safe_statics@@YAXXZ 00000001800062e0     MSVCRT:thread_safe_statics.obj
 0002:000022e0       $unwind$__scrt_acquire_startup_lock 00000001800062e0     MSVCRT:utility.obj
 0002:000022e0       $unwind$__scrt_dllmain_after_initialize_c 00000001800062e0     MSVCRT:utility.obj
 0002:000022e0       $unwind$__scrt_dllmain_before_initialize_c 00000001800062e0     MSVCRT:utility.obj
 0002:000022e0       $unwind$__scrt_dllmain_crt_thread_attach 00000001800062e0     MSVCRT:utility.obj
 0002:000022e0       $unwind$__scrt_dllmain_crt_thread_detach 00000001800062e0     MSVCRT:utility.obj
 0002:000022e0       $unwind$__scrt_dllmain_uninitialize_c 00000001800062e0     MSVCRT:utility.obj
 0002:000022e0       $unwind$__scrt_dllmain_uninitialize_critical 00000001800062e0     MSVCRT:utility.obj
 0002:000022e0       $unwind$atexit             00000001800062e0     MSVCRT:utility.obj
 0002:000022e8       $unwind$nsk_jvmti_lverify  00000001800062e8     libretransform004.obj
 0002:000022fc       $unwind$exitOnError        00000001800062fc     libretransform004.obj
 0002:0000230c       $unwind$Java_nsk_share_jvmti_ArgumentHandler_getAgentOptionsString 000000018000630c     libretransform004.obj
 0002:00002320       $unwind$Java_nsk_jvmti_unit_FollowReferences_FollowRefObjects_getTag 0000000180006320     libretransform004.obj
 0002:00002320       $unwind$Java_nsk_share_jvmti_DebugeeClass_checkStatus 0000000180006320     libretransform004.obj
 0002:00002320       $unwind$agentThreadWrapper 0000000180006320     libretransform004.obj
 0002:00002330       $unwind$startAgentThreadWrapper 0000000180006330     libretransform004.obj
 0002:0000234c       $unwind$syncDebuggeeStatus 000000018000634c     libretransform004.obj
 0002:0000234c       $unwind$__scrt_dllmain_exception_filter 000000018000634c     MSVCRT:utility.obj
 0002:00002360       $unwind$Java_nsk_share_jvmti_DebugeeClass_resetAgentData 0000000180006360     libretransform004.obj
 0002:00002368       $unwind$MA_checkStatus     0000000180006368     libretransform004.obj
 0002:0000237c       $unwind$Java_nsk_jvmti_unit_FollowReferences_FollowRefObjects_setTag 000000018000637c     libretransform004.obj
 0002:00002394       $unwind$Java_nsk_jvmti_unit_FollowReferences_FollowRefObjects_addRefToVerify 0000000180006394     libretransform004.obj
 0002:000023b0       $unwind$Agent_Initialize   00000001800063b0     libretransform004.obj
 0002:000023d0       $unwind$Java_nsk_jvmti_RetransformClasses_retransform004_forceLoadedClassesRetransformation 00000001800063d0     libretransform004.obj
 0002:000023dc       $unwind$ClassFileLoadHook  00000001800063dc     libretransform004.obj
 0002:000023f4       $unwind$capture_previous_context 00000001800063f4     MSVCRT:gs_report.obj
 0002:00002400       $unwind$__GSHandlerCheckCommon 0000000180006400     MSVCRT:gshandler.obj
 0002:00002408       $xdatasym                  0000000180006408     MSVCRT:amdsecgs.obj
 0002:0000240c       $unwind$?dllmain_crt_process_attach@@YAHQEAUHINSTANCE__@@QEAX@Z 000000018000640c     MSVCRT:dll_dllmain.obj
 0002:00002448       $unwind$?fin$0@?0??dllmain_crt_process_attach@@YAHQEAUHINSTANCE__@@QEAX@Z@4HA 0000000180006448     MSVCRT:dll_dllmain.obj
 0002:00002448       $unwind$?fin$0@?0??dllmain_crt_process_detach@@YAH_N@Z@4HA 0000000180006448     MSVCRT:dll_dllmain.obj
 0002:00002448       $unwind$?fin$1@?0??dllmain_crt_process_detach@@YAH_N@Z@4HA 0000000180006448     MSVCRT:dll_dllmain.obj
 0002:00002450       $unwind$?dllmain_crt_process_detach@@YAH_N@Z 0000000180006450     MSVCRT:dll_dllmain.obj
 0002:000024a4       $unwind$?dllmain_dispatch@@YAHQEAUHINSTANCE__@@KQEAX@Z 00000001800064a4     MSVCRT:dll_dllmain.obj
 0002:000024cc       $unwind$?filt$0@?0??dllmain_dispatch@@YAHQEAUHINSTANCE__@@KQEAX@Z@4HA 00000001800064cc     MSVCRT:dll_dllmain.obj
 0002:000024d4       $unwind$_DllMainCRTStartup 00000001800064d4     MSVCRT:dll_dllmain.obj
 0002:000024e4       $unwind$__scrt_is_nonwritable_in_current_image 00000001800064e4     MSVCRT:utility.obj
 0002:00002504       $unwind$__scrt_is_nonwritable_in_current_image$filt$0 0000000180006504     MSVCRT:utility.obj
 0002:0000250c       $unwind$__scrt_fastfail    000000018000650c     MSVCRT:utility_desktop.obj
 0002:0000251c       $unwind$__security_init_cookie 000000018000651c     MSVCRT:gs_support.obj
 0002:00002528       $unwind$__isa_available_init 0000000180006528     MSVCRT:cpu_disp.obj
 0002:00002538       $xdatasym                  0000000180006538     MSVCRT:guard_dispatch.obj
 0002:00002540       $xdatasym                  0000000180006540     MSVCRT:guard_xfg_dispatch.obj
 0002:00002550       .edata                     0000000180006550     retransform004.exp
 0002:00002578       rgpv                       0000000180006578     retransform004.exp
 0002:000025b4       rgszName                   00000001800065b4     retransform004.exp
 0002:000025f0       rgwOrd                     00000001800065f0     retransform004.exp
 0002:0000260e       szName                     000000018000660e     retransform004.exp
 0002:00002621       $N00001                    0000000180006621     retransform004.exp
 0002:00002630       $N00002                    0000000180006630     retransform004.exp
 0002:0000263d       $N00003                    000000018000663d     retransform004.exp
 0002:00002691       $N00004                    0000000180006691     retransform004.exp
 0002:000026d6       $N00005                    00000001800066d6     retransform004.exp
 0002:00002713       $N00006                    0000000180006713     retransform004.exp
 0002:0000275b       $N00007                    000000018000675b     retransform004.exp
 0002:0000279b       $N00008                    000000018000679b     retransform004.exp
 0002:000027d8       $N00009                    00000001800067d8     retransform004.exp
 0002:00002813       $N00010                    0000000180006813     retransform004.exp
 0002:00002841       $N00011                    0000000180006841     retransform004.exp
 0002:00002872       $N00012                    0000000180006872     retransform004.exp
 0002:000028a1       $N00013                    00000001800068a1     retransform004.exp
 0002:000028d0       $N00014                    00000001800068d0     retransform004.exp
 0002:00002905       $N00015                    0000000180006905     retransform004.exp
 0002:00002d0a       .idata$6                   0000000180006d0a     kernel32:KERNEL32.dll
 0002:00002d6e       .idata$6                   0000000180006d6e     vcruntime:VCRUNTIME140.dll
 0002:00002ed0       .idata$6                   0000000180006ed0     ucrt:api-ms-win-crt-runtime-l1-1-0.dll
 0002:00002ef2       .idata$6                   0000000180006ef2     ucrt:api-ms-win-crt-stdio-l1-1-0.dll
 0002:00002f12       .idata$6                   0000000180006f12     ucrt:api-ms-win-crt-string-l1-1-0.dll
 0003:00000000       ?codeAttributeName@@3PEBDEB 0000000180007000     libretransform004.obj
 0003:00000008       ?lineNumberAttributeName@@3PEBDEB 0000000180007008     libretransform004.obj
 0003:00000010       ?localVarAttributeName@@3PEBDEB 0000000180007010     libretransform004.obj
 0003:00000018       ?localVarTypeAttributeName@@3PEBDEB 0000000180007018     libretransform004.obj
 0003:00000020       ?stackMapAttributeName@@3PEBDEB 0000000180007020     libretransform004.obj
 0003:00000028       ?callBytes@@3PAEA          0000000180007028     libretransform004.obj
 0003:0000002c       ?allocBytes@@3PAEA         000000018000702c     libretransform004.obj
 0003:0001aad4       redefineAttempted          0000000180021ad4     libretransform004.obj
 0003:0001aad8       nsk_context                0000000180021ad8     libretransform004.obj
 0003:0001aae4       redefineSucceed            0000000180021ae4     libretransform004.obj
 0003:0001aae8       agentFailed                0000000180021ae8     libretransform004.obj
 0003:0001aaec       currentAgentStatus         0000000180021aec     libretransform004.obj
 0003:0001aaf0       context                    0000000180021af0     libretransform004.obj
 0003:0001aba8       agentThread                0000000180021ba8     libretransform004.obj
 0003:0001abb0       agentThreadProc            0000000180021bb0     libretransform004.obj
 0003:0001abb8       agentThreadArg             0000000180021bb8     libretransform004.obj
 0003:0001abc0       agent_data                 0000000180021bc0     libretransform004.obj
 0003:0001abd0       jvmti_env                  0000000180021bd0     libretransform004.obj
 0003:0001abd8       jvm                        0000000180021bd8     libretransform004.obj
 0003:0001abe0       jni_env                    0000000180021be0     libretransform004.obj
 0003:0001abe8       checkStatus_func           0000000180021be8     libretransform004.obj
 0003:0001abf0       ?codeAttributeIndex@@3GA   0000000180021bf0     libretransform004.obj
 0003:0001abf4       ?lineNumberAttributeIndex@@3GA 0000000180021bf4     libretransform004.obj
 0003:0001abf8       ?localVarAttributeIndex@@3GA 0000000180021bf8     libretransform004.obj
 0003:0001abfc       ?localVarTypeAttributeIndex@@3GA 0000000180021bfc     libretransform004.obj
 0003:0001ac00       ?stackMapAttributeIndex@@3GA 0000000180021c00     libretransform004.obj
 0003:0001ac04       ?stackFrameOffset@@3GA     0000000180021c04     libretransform004.obj
 0003:0001ac08       ?mode@@3HA                 0000000180021c08     libretransform004.obj
 0003:0001ac0c       ?constantPoolSize@@3GA     0000000180021c0c     libretransform004.obj
 0003:0001ac10       ?orig@@3PEBEEB             0000000180021c10     libretransform004.obj
 0003:0001ac18       ?gen@@3PEAEEA              0000000180021c18     libretransform004.obj
 0003:0001ac20       ?inputPos@@3PEAEEA         0000000180021c20     libretransform004.obj
 0003:0001ac28       ?endPos@@3PEBEEB           0000000180021c28     libretransform004.obj
 0003:0001ac30       ?genPos@@3PEAEEA           0000000180021c30     libretransform004.obj
 0003:0001ac38       ?markPos@@3PEAEEA          0000000180021c38     libretransform004.obj
 0003:0001ac40       ?constantPool@@3PEAPEADEA  0000000180021c40     libretransform004.obj
 0003:0001ac48       ?constantPoolCount@@3GA    0000000180021c48     libretransform004.obj
 0003:0001ac4c       ?zeroBytes@@3PAEA          0000000180021c4c     libretransform004.obj
 0003:0001ac50       ?codeLength@@3IA           0000000180021c50     libretransform004.obj
 0003:0001ac58       ?map@@3PEAIEA              0000000180021c58     libretransform004.obj
 0003:0001ac60       ?widening@@3PEACEA         0000000180021c60     libretransform004.obj
 0003:0001ac68       jvmti                      0000000180021c68     libretransform004.obj
 0003:0001ac80       GS_ExceptionRecord         0000000180021c80     MSVCRT:gs_report.obj
 0003:0001ad20       GS_ContextRecord           0000000180021d20     MSVCRT:gs_report.obj
 0003:0001b1f0       ?g_tss_cv@@3U_RTL_CONDITION_VARIABLE@@A 00000001800221f0     MSVCRT:thread_safe_statics.obj
 0003:0001b1f8       ?g_tss_event@@3PEAXEA      00000001800221f8     MSVCRT:thread_safe_statics.obj
 0003:0001b200       ?g_tss_mutex@@3U_RTL_CRITICAL_SECTION@@A 0000000180022200     MSVCRT:thread_safe_statics.obj
 0003:0001b228       ?g_sleep_condition_variable_cs@@3P6AHPEAU_RTL_CONDITION_VARIABLE@@PEAU_RTL_CRITICAL_SECTION@@K@ZEA 0000000180022228     MSVCRT:thread_safe_statics.obj
 0003:0001b230       ?g_wake_all_condition_variable@@3P6AXPEAU_RTL_CONDITION_VARIABLE@@@ZEA 0000000180022230     MSVCRT:thread_safe_statics.obj
 0003:0001b23c       ?__proc_attached@@3HA      000000018002223c     MSVCRT:dll_dllmain.obj
 0003:0001b250       ?is_initialized_as_dll@@3_NA 0000000180022250     MSVCRT:utility.obj
 0003:0001b251       ?module_local_atexit_table_initialized@@3_NA 0000000180022251     MSVCRT:utility.obj
 0003:0001b258       ?module_local_atexit_table@@3U_onexit_table_t@@A 0000000180022258     MSVCRT:utility.obj
 0003:0001b270       ?module_local_at_quick_exit_table@@3U_onexit_table_t@@A 0000000180022270     MSVCRT:utility.obj
